:0400000000000428D0
:080008008A110A120728E130F9
:100010008316031386008501912083128C1E0D2800
:100020001A0883120313AD0031302D02031C3D2842
:1000300035302D0203183D28CF30AD0700308A003F
:1000400025302D0703188A0A820029282E283328F4
:10005000382802308312031386060D2804308312D9
:10006000031386060D2808308312031386060D2815
:1000700010308312031386060D28EB30831203130E
:1000800086050D28080083120313A8007F08A70027
:10009000A90129082707AA002808AB000318AB0A02
:1000A0002A0884000008AC0003195C282C087D2075
:1000B00083120313A90A4928080083120313A2001C
:1000C0007F08A100A30123082107A4002208A5009E
:1000D0000318A50A6F2825088A00240882006B20CF
:1000E00083120313A600260803197C2826087D2006
:1000F00083120313A30A6328080083120313A000CA
:10010000831203130C1E802883120313200883120A
:10011000031399000800831203138C1E8B281A08FE
:100120000800813083160313990024309800903022
:0601300083129800080094
:02400E00FF3F72
:00000001FF
